:020000020000FC
:1000000010C085C099C099C0CAC0C4C0C1C0C1C019
:10001000C2C094C094C094C0C0C0C0C0BDC0C0C065
:10002000C0C0F89400E811E006BD16BD00E00BBBAF
:100030000FEF0ABB0CE008BB03EF07BBB0E0A0E684
:1000400000E00D93B130E9F7A036D9F711E00FE5E4
:100050001EBF0DBF00E000B901E005BF00E000BF1A
:1000600001E003BF00E006BF00E00CBF00E003BDFD
:1000700000E00FBD03E20EBD00E002BD10E000E0B5
:100080001DBD0CBD10E000E01BBD0ABD10E000E08E
:1000900019BD08BD10E000E015BD04BD00E007B9C2
:1000A00000E006B900E103B900E001B900E808B9D1
:1000B000A89504B7077F04BF09E319E301BD11BD8B
:1000C00000E70ABF07E008BF07E20BB900E002BB88
:1000D00000E000BD00E40BBF01E009BF00E00CB987
:1000E00000E0102E00E0302E0DE5202E00E0502E16
:1000F0000DE5402E00E0602E00E0702E90E0789438
:10010000A89590FFFDCF9E7F422C532CF9CFFFB6D0
:100110000F93B29907C000E00EBD1DBC1CBC03E2EA
:100120000EBD07C000E00EBD2CB43DB403E20EBD11
:1001300091600F91FFBE1895189518951895189510
:10014000FFB60F931F93739441F0761409F01CC00F
:1001500000E00BBB0CE008BB17C0F2E0E0E0E40DF0
:10016000F11DEE0FFF1FC895002D3196C895102D7B
:100170000BBB18BBF3E0E0E0E40DF11DEE0FFF1F39
:10018000C895602C916000C01F910F91FFBE18951B
:1001900018951895189518951895189518951895F7
:1001A000189518951F932F932BE111E31A95F1F7EA
:0E01B0002A95D9F70A95C1F72F911F9108954E
:10040000000C000C000C000C000C000C000C000C8C
:10041000000C000C000C000C000C000C000C000C7C
:10042000000C000C000C000C000C000C000C000C6C
:10043000000C000C000C000C000C000C000C000C5C
:10044000000C000C000C000C000C100C100C100C1C
:10045000100C100C100C100C100C100C100C100CBC
:10046000100C100C100C100C100C100C100C100CAC
:10047000100C100C100C100C100C100C100C100C9C
:10048000100C100C100C100C100C100C100C100C8C
:10049000180C180C180C180C180C1C0C1C0C1C0C30
:1004A0001C0C1C0C1E0C1E0C1E0C1E0C1E0C1F0CFF
:1004B0001F0C1F0C1F0C1F0C000C000C000C000C60
:1004C000E00FE00FE00FE00FE00FE00EE00EE00EB7
:1004D000E00EE00EE00CE00CE00CE00CE00CC00CD8
:1004E000C00CC00CC00CC00C800C800C800C800CAC
:1004F000800C800C800C800C800C800C800C800C9C
:10050000800C800C800C800C800C800C800C800C8B
:10051000800C800C800C800C800C800C800C800C7B
:10052000800C800C800C800C800C800C800C800C6B
:10053000800C800C800C800C800C000C000C000CDB
:10054000000C000C000C000C000C000C000C000C4B
:10055000000C000C000C000C000C000C000C000C3B
:10056000000C000C000C000C000C000C000C000C2B
:10057000000C000C000C000C000C000C000C000C1B
:10058000000C000C000C000C000C000C000C000C0B
:10059000000C000C000C000C000C000C000C000CFB
:1005A000000C000C000C000C000C000C000C000CEB
:1005B000000C000C000C000C000C000C000C000CDB
:1005C000000C000C000C000C000C000C000C000CCB
:1005D000000C000C000C000C000C000C000C000CBB
:1005E000000C000C000C000C000C000C000C000CAB
:1005F000000C000C000C000C000C000C000C000C9B
:1006000000000000000000000000000000000000EA
:1006100000000000000000000000000000000000DA
:1006200000000000000000000000000000000000CA
:1006300000000000000000000000000000000000BA
:1006400000000000000000000000FF00FF00FF00AD
:10065000FF00FF00FF00FF00FF00FF00FF00FF00A2
:10066000FF00FF00FF00FF00FF00FF00FF00FF0092
:10067000FF00FF00FF00FF00FF00FF00FF00FF0082
:10068000FF00FF00FF00FF00FF00FF00FF00FF0072
:10069000CD00CD00CD00CD00CD009A009A009A008B
:1006A0009A009A00660066006600660066003300E5
:1006B000330033003300330000000000000000006E
:1006C00033003300330033003300660066006600F9
:1006D000660066009A009A009A009A009A00CD007F
:1006E000CD00CD00CD00CD00FF00FF00FF00FF00DA
:1006F000FF00FF00FF00FF00FF00FF00FF00FF0002
:10070000FF00FF00FF00FF00FF00FF00FF00FF00F1
:10071000FF00FF00FF00FF00FF00FF00FF00FF00E1
:10072000FF00FF00FF00FF00FF00FF00FF00FF00D1
:10073000FF00FF00FF00FF00FF00000000000000BE
:1007400000000000000000000000000000000000A9
:100750000000000000000000000000000000000099
:100760000000000000000000000000000000000089
:100770000000000000000000000000000000000079
:100780000000000000000000000000000000000069
:100790000000000000000000000000000000000059
:1007A0000000000000000000000000000000000049
:1007B0000000000000000000000000000000000039
:1007C0000000000000000000000000000000000029
:1007D0000000000000000000000000000000000019
:1007E0000000000000000000000000000000000009
:1007F00000000000000000000000000000000000F9
:00000001FF
